:020000040000FA
:02000000822854
:040002000034003492
:020008000528C9
:06000A0081010B118B10B7
:10001000051D08280B1D7F280514A101A0010C3027
:10002000A2000519112881016400051D1528010889
:100030008F3EA10CA00CA20B11280310A10CA00C48
:10004000A10CA00CA10CA00C0310A00C21080E3ACE
:10005000031D7F28A3142008193A031D3D28231CE3
:100060003B282411831607118312071181010B11FC
:100070000B1D38282310A4117028231020081B3AC8
:10008000031D44282410702820081C3A031D4A2808
:10009000A41070282008183A031D5028A4127028B4
:1000A0002008203A031D5B28851E7F28051A662834
:1000B000A3122514752820081A3A031D6A28851EE4
:1000C0006628051E662823122514752825187F2802
:1000D0002412702820081E3A031D7F28241123149F
:1000E00024088316870083128700230883163C396F
:1000F00085008312230885008E018F010C108B1060
:100100008B170900831603308E003F3087003C3088
:10011000850082308100FF23900083120730990010
:100120003530900090308B00A5013C30A3003F306B
:10013000A400870085008E018F010C1064000C1C48
:100140009E280C103F308700A4003C3023183D301F
:100150008500A30083163F3087003C308500831262
:04016000A5019E282F
:02400E00BC3FB5
:00000001FF
